:1000000012C0189518951895189518951895189563
:100010001895189518951895189518951895189578
:100020001895189518958FE58DBFC0E4E0E44E2E25
:1000300084E08EBFD4E0F4E05F2EEEEFF3E0A0E6C4
:10004000B0E088278D933197E9F7B3D16624E6E6CF
:10005000F0E080E4F6D158E0C895802DECD13196DF
:100060005A95D1F704C020201F1F1F1F2020E6E84B
:10007000F0E088E4E6D158E0C895802DDCD13196D7
:100080005A95D1F704C00101010101010101E6EA1D
:10009000F0E080E5D6D158E0C895802DCCD13196DE
:1000A0005A95D1F704C01010101010101010E6EC83
:1000B000F0E088E5C6D158E0C895802DBCD13196D6
:1000C0005A95D1F704C010101F1F1F1F1010E6EE25
:1000D000F0E080E6B6D158E0C895802DACD13196DD
:1000E0005A95D1F704C001011F1F1F1F0101E6E04F
:1000F000F1E088E6A6D158E0C895802D9CD13196D4
:100100005A95D1F704C020201C1C1C1C202086E01E
:1001100086B980E487B9379A38D18CE092D183E9E7
:1001200011E042D1E4EDF5E02AD183E915E03CD1BC
:10013000E6EDF5E024D183E91AE036D1EAEDF5E009
:100140001ED183E91FE030D1EEEDF5E018D183E94F
:1001500013E12AD18FED6FD1E2EEF5E010D180E40A
:10016000806487B9B3D1A0E6B0E08D939C93A0E6FC
:10017000B0E00D911C9145E050E09ED1A4E6B0E0C6
:100180000D931C93009164004AE014D2A6E6B0E0FF
:100190008C93A4E6B0E00D911C914AE050E0CDD0E4
:1001A000A4E6B0E04D935C938FE711E0FDD0A8E2A8
:1001B000B4E0E4E6F0E0A5D1DAD0E4EEF5E0DFD09B
:1001C000A8E2B4E0E6E6F0E0ABD1D1D00091640063
:1001D00042E0F0D1A9E6B0E00C938FEB11E0E4D05F
:1001E00081E08093680040916900009168000417E5
:1001F00010F009F029C000916800013009F003C037
:1002000083E019D11AC0053009F003C084E013D18E
:1002100014C00A3009F003C084E00DD10EC00F30C5
:1002200009F003C084E007D108C0043109F003C01D
:1002300084E001D102C080E0FED0A8E6B0E08C915D
:100240008F5F8C9308F4CFCF0091690042E0B2D168
:10025000AAE6B0E08C9300916A00003010F009F03B
:1002600001C008C085E0E7D0A9E6B0E08C918E5FC0
:100270008C9305C0A9E6B0E08C918F5F8C93809140
:1002800069008093680000916800043110F009F063
:1002900029C000916800013009F003C082E0CBD092
:1002A0001AC0053009F003C081E0C5D014C00A307F
:1002B00009F003C081E0BFD00EC00F3009F003C0C9
:1002C00081E0B9D008C0043109F003C081E0B3D0A7
:1002D00002C080E2B0D0A8E6B0E08C918F5F8C9332
:1002E00008F4D1CF88EE93E0D8D039CFF894FFCF7F
:1002F00008D0E2D000FC10D0089503D01ED001F841
:10030000F9CF0024E89457FF02C009D0689400F8A0
:100310000BD010F80124089502D009D0089550950B
:1003200040954F5F5F4F0895E89417FF089500953B
:1003300010950F5F1F4F68940895352F242FE89470
:10034000452B11F468940895512F402F0027112751
:1003500080E1440F551F001F111F021B130B41604A
:1003600018F4020F131F4E7F8A9599F70895A8E29B
:10037000B4E08D91882311F05ED0FBCF0895AFD00B
:10038000802D11F058D0FBCF089581E05AD00ED0C7
:1003900080E857C08FE7213039F08FEB223021F011
:1003A00083E9233009F083ED810F4BC083E0992767
:1003B00074C08AEF90E071D0889A899A8A9A8B9A51
:1003C0008E9A8F9A979885E090E067D0969890984B
:1003D0009198929A939A969AEF93FF93E6EFF0E0B2
:1003E00050D0FF91EF91969855D0969AEF93FF9346
:1003F000E6EFF0E046D0FF91EF9196984BD0969AB9
:10040000EF93FF93E6EFF0E03CD0FF91EF919698E9
:1004100041D09398969AEF93FF93E6EFF0E031D0B6
:10042000FF91EF91969836D088E20BD08EE009D0FC
:1004300086E007D00895979A829505D004D02AD0F7
:1004400008959798F9CF859510F4939A01C09398E1
:10045000859510F4929A01C09298859510F4919A1E
:1004600001C09198859510F4909A01C09098969A41
:10047000EF93FF93E6EFF0E004D0FF91EF919698B1
:1004800008953197F1F70895689462F80895E89413
:1004900062F8089581E090E000C0EF93FF93EE27AB
:1004A000E82BE92B31F0E4ECF9E03197F1F7019713
:1004B000D1F7FF91EF9108950F92B801469F800107
:1004C000479F100D569F100D0F900895369A36993C
:1004D000FECF369A3699FECF84B195B10895C8956E
:1004E000319600200895000F111F221F331F089519
:1004F00000951095209530950F5F1F4F2F4F3F4F60
:100500000895019110810EC00191119121913081C6
:100510000BC00191108117FF05C03FEF2FEF04C002
:10052000008111272227332737FF03C0E1DF8DE247
:100530008D93CF93DF93CF92DF92EF92AA24BB24C7
:10054000CC24DD24EE2440E2CAE0DD2755E093E32D
:100550008881890F87FD9F7083FD907F891B899318
:100560005A95A9F7C0DFAA1CBB1CCC1CDD1CEE1CD5
:100570004A9551F7E894EFE0FF2782910ED0EB30D7
:10058000E0F71EF068948A2D0CD088278D93EF90A9
:10059000DF90CF90DF91CF910895982F829501D071
:1005A000892F8F70805D26F0803309F40895689458
:1005B0008D930895FF93881BF9E0001FFA9511F4BD
:1005C000FF910895881F841B18F4840F8894F5CF39
:1005D0000894F3CF30003130000032300000333067
:0605E000000043002C00A6
:00000001FF
